:020000040000FA
:0400000000EF04F019
:0400080004EF04F00D
:040018000CEF04F0F5
:040800000EEF04F003
:0408080004EF04F005
:080818000CEF04F0070EB46EB2
:10082000000E896E000E8A6E400E8B6E000E8C6E6E
:10083000CC0E8D6E000E8E6E020E8F6EFF0E926EBF
:10084000FF0E936EBF0E946EFF0E956E330E966E76
:10085000FF0E976EFD0E986E0F0EC16E0C0EAF6EF2
:10086000AC84AC8AAB88AB8E0C0E6F6E6C846C8AD9
:100870006B886B8E8D9C04D800D08D8C01D8FAD7F4
:10088000340E026E450E016E8A0E006E002EFED7EB
:10089000012EFAD7022EF6D71200A4A8FED76D6E4D
:1008A00012006BA202D06B986B88A4AAFED76E5080
:0208B000120034
:020000040030CA
:06000100061600F38381E6
:06000800FF80FF80FF00F5
:00000001FF
